:100000000207F5C0E0C0D075D000C000781C06E63D
:0D00100018700106C2CFD000D0D0D0E03271
:030023000208814F
:03002B00020003CD
:10003300020036C0E0C0F0C083C082C0D075D000DB
:10004300C000C001C002C003C004C005C006C00791
:1000530030FC05C2FC0202AD85A315E521B40E00F8
:1000630040030202A890006FF82828730200990247
:10007300010E02011702012902013C02022E0202B3
:10008300A802028702028902029A0201AB0201B5A9
:100093000201BB0201EFE51524BF604224EC60249A
:1000A30024FA601B24B8602214602514602A24FB00
:1000B3006020245060030202AB7521010202AB757C
:1000C3002801805C7521040202AB7521090202AB91
:1000D30080337521080202AB852AA30202A3751699
:1000E300FF7517097518D2AB16AA17A9181203BE04
:1000F30060130518E5187002051714F91203BEFF03
:1001030012075380E28529A30202A38515227521D4
:10011300020202AB851528E5287005F5210202AB22
:100123007521030202ABAF151207531528E52860AA
:10013300030202ABF5210202AB851522120A3E8EA1
:10014300268F27D3EF9400EE94004056D3E52794EF
:1001530008E52694004006752600752708AF27EFAB
:10016300F5A3752500E522640270318F25F52BF583
:100173002CF515E515C39525501C1203FD74312587
:1001830015F8A60774312515F8E6252CFF752B0005
:100193008F2C051580DD75210A0202AB752105023E
:1001A30002AB75A3000202A8E525F4F5A3752E00A2
:1001B300803475210C0202ABE515B406030202A8D4
:1001C300E515B4181B751500E515C39525500E7478
:1001D300312515F8E6FF120A61051580EB0202A826
:1001E3008531A3752E0175210D0202ABE515B418F7
:1001F3001B751500E515C39525500E74312515F8AB
:10020300E6FF120A61051580EB0202A8E52EC395ED
:1002130025500EAF2E052E74312FF8E6F5A30202FA
:10022300ABE52CF4F5A375210B807DE515B4181A05
:10023300751500E515C39525500E74312515F8E69F
:10024300FF120A61051580EB805BD3E5279400E577
:10025300269400402D1203FD8F158515A3AF2505A8
:100263002574312FF8A615E525C394094003752598
:1002730008E527152770021526144526702AF5214F
:1002830080268021801F532AF8E5155437422A75AA
:100293002300752400800EAF151205098F298FA343
:1002A3007521078003752100C2FFD007D006D00552
:1002B300D004D003D002D001D000D0D0D082D083DC
:1002C300D0F0D0E032E709F608DFFA8046E709F21A
:1002D30008DFFA803E88828C83E709F0A3DFFA8087
:1002E30032E309F608DFFA8078E309F208DFFA80DF
:1002F3007088828C83E309F0A3DFFA806489828AA1
:1003030083E0A3F608DFFA805889828A83E0A3F2A8
:1003130008DFFA804C80D280FA80C680D48069805E
:10032300F28033801080A680EA809A80A880DA80E9
:10033300E280CA803389828A83ECFAE493A3C8C536
:1003430082C8CCC583CCF0A3C8C582C8CCC583CC36
:10035300DFE9DEE7800D89828A83E493A3F608DF71
:10036300F9ECFAA9F0EDFB2289828A83ECFAE0A387
:10037300C8C582C8CCC583CCF0A3C8C582C8CCC5C8
:1003830083CCDFEADEE880DB89828A83E493A3F20D
:1003930008DFF980CC88F0EF60010E4E60C388F06F
:1003A300ED2402B4040050B9F582EB2402B4040036
:1003B30050AF232345822390031873BB0106898220
:1003C3008A83E0225002E722BBFE02E32289828A6B
:1003D30083E49322D083D082F8E493701274019360
:1003E300700DA3A393F8740193F5828883E4737467
:1003F30002936860EFA3A3A380DFD3793BE7783F41
:100403009619E71896500F9001DAE0FF9001D9E0B2
:100413009F50037FFF229001DAE0FF9001D9E0FEB5
:10042300D39F405DA3E004F074DB2FF582E4340135
:10043300F583E0F5199001DAE0FFB5060AE49001CF
:10044300D9F0A3F0020500EFD3940F500302050087
:100453009001D9E0FFA3E0FEEF9E9001D9F0F58271
:1004630075830074DB2EF9E43401FA7B0178DB7CBD
:10047300017D017E00AF82120398E49001DAF080DF
:100483007CE49001D9F0A3F0783AE6FE08E6FFD3C6
:10049300783F96EE1896405A0806E61886047001CF
:1004A30006142401F58274003CF583E0F519783EC7
:1004B300E6FC08E6FDB5070CECB50608E4783AF669
:1004C30008F6802AD3ED946AEC94004030783BE63A
:1004D3009DFF18E69CFEF608EFF674012DF97400F3
:1004E3003CFA7B0178017C007D01120398E4783E9D
:1004F3008008E4783EF608F6783AF608F6D292D207
:1005030094D293AF19228F19538EF4E519C394250E
:100513004066C2CA75B28375CB9C75CA4FD2CAE511
:10052300191203D7054604054B0905501205552535
:10053300055738055C4B056170056696056BE10050
:10054300000573758D2B805F758D96805A758DCBE5
:100553008055801F758DB8806D758DCB8068758DC6
:10056300968056758DB08051758D2B438E088056BD
:10057300751925758D96804EC2CA75B28075CB3CB0
:1005830075CAB0D2CAE51924FE601924FE601D2481
:10059300FB601E24F7601F24ED6023242470217563
:1005A3008D968003758DCB438E02801A758D6A807C
:1005B30015758D608003758DB0438E0180088003AF
:1005C300751925758DA0D200D202C201E4783AF6DE
:1005D30008F69001D9F008F608F67840F608F678A0
:1005E3003EF608F6A3F0AF19221209507BFF7A09F1
:1005F300799A120A197BFF7A0979AD120A19C297FF
:10060300D290E4781BF608F6C3781CE6942818E623
:10061300940040F4D2977BFF7A0979C1120A191228
:100623000AE8E4F52A752DFFD2AED2BE75ECFF12AF
:100633000A3ED3EF9400EE94004005432A0880035A
:10064300532AF7781BE6FE08E6FF65307003EE6574
:100653002F600C8E2F8F300524E52470020523C3F1
:10066300EF9450EE94004006E4781BF608F6C3E5D9
:100673002494C8E5239400400F7523007524C8D241
:1006830090D297532ACF801EC3E5249464E5239424
:10069300004007D297532AEF800CE52A30E407C2C3
:1006A3009730E502C290852A2D80818F14D378413B
:1006B300E6940018E694004059D2017840E6FE081B
:1006C300E6FF783CE6FC08E6FDD39FEC9E500AE487
:1006D3007840F608F6783C8034C3EF944BEE9400F0
:1006E300402EED784196793DF7EC189619F7783C52
:1006F300E6FE08E6FF7841E62442F9E43401FA7B9A
:100703000178427C017D01120398E47840F608F6F3
:10071300C201C3783DE6949518E6940040107841F1
:10072300E6184670943002F6C202D29980F0783C03
:100733000806E6188606700106142442F582740141
:100743003EF583E514F0300204C202D299AF1422BD
:100753008F197840E6FE08E6FFD39400EE9400403C
:1007630052D201783CE6FC08E6FDD39FEC9E500A8A
:10077300E47840F608F6783C8034C3EF944BEE946B
:1007830000402EED784196793DF7EC189619F778ED
:100793003CE6FE08E6FF7841E62442F9E43401FA38
:1007A3007B0178427C017D01120398E47840F608CE
:1007B300F6C201C3783DE6949518E694004011789B
:1007C30041E618467007300204C202D2997F002224
:1007D300783C0806E6188606700106142442F58262
:1007E30074013EF583E519F0300204C202D2997F09
:1007F3000122787FE4F6D8FD75814102083C0205A9
:10080300ECE493A3F8E493A34003F68001F208DF3A
:10081300F48029E493A3F85407240CC8C333C454C5
:100823000F4420C8834004F456800146F6DFE48079
:100833000B0102040810204080900AABE47E019370
:1008430060BCA3FF543F30E509541FFEE493A3604B
:10085300010ECF54C025E060A840B8E493A3FAE4A6
:1008630093A3F8E493A3C8C582C8CAC583CAF0A3F7
:10087300C8C582C8CAC583CADFE9DEE780BEC0E057
:10088300C083C082C0D075D00830982FC298C37877
:100893003BE6943F18E6940150150806E618860EC9
:1008A300700106142401F58274003EF5838009C2A9
:1008B30092C294C293900000E599F0309932C299A4
:1008C30020012BD3793DE778419619E71896401814
:1008D3000806E618860E700106142442F582740198
:1008E3003EF583E0F5998002D202D2008002D20263
:1008F300D0D0D082D083D0E032C299C28EC2AB7541
:100903009810D29CC2CA75B28375CB9C75CA4FD25C
:10091300CA758D96538EF4D200D202C201E4783A9E
:10092300F608F69001D9F008F608F67840F608F6CE
:10093300783EF608F6A3F0758BFF53890F438920A1
:10094300C299C298D2ACD2BCD299D28E2253D9BF0B
:10095300E4F5A8F5B8F5E6F5F675E477D297120A4B
:10096300E175D90275EBFF75ECFF120AD0120A7B11
:10097300120A941208FCE4F510120ABE0510E510E1
:10098300C3946440F4D2AFE4F510120ABE0510E537
:1009930010C3946440F42220202020202020202013
:1009A300202020202020200D0A0044333030452011
:1009B30033333120537461727475700D0A004433FC
:1009C30030304520333331204C6F6F700D0A0044B3
:1009D300333030452033333120546573740D0A00AE
:1009E3008F13E513D3947F40037F0022E513B40AEA
:1009F300057F0D1206AEE513C394205011E51324B1
:100A0300F824FD500924FE600580007F0022AF1307
:100A13001206AEAF13228B108A118912AB10AA11E2
:100A2300A9121203BE60130512E512700205111418
:100A3300F91203BEFF1209E380E2229001DAE0FF1C
:100A43009001D9E0C39FFFE49400FEC3793BE778AC
:100A53003F96FD19E71896CD2FFFED3EFE2290013C
:100A6300D9E0C3941D5010E0FE04F074DB2EF58230
:100A7300E43401F583EFF02275A45475A5F475F100
:100A8300FF75F2FFE4F5D475D5FF75E10B75E24010
:100A930022E4F5C8538ECF75CB9E75CA5874FFF503
:100AA300CDF5CCD2ADD2CA22012925022F000002F6
:100AB300230000012100021B000000E4FFFE75EC8F
:100AC300FF0FBF00010EBE01F5BFF4F22275A20BAA
:100AD30075A10775F804D2F9E4F5A3D2F822E4F579
:0C0AE300A975B28322E4783AF608F622E6
:00000001FF
